:020000040000FA
:060000000219FD0200C818
:03000B0002008D63
:03002B000200923E
:03005B000202CDD1
:030073000200B5D3
:100080000406080C10182030406080A0C0C28D0506
:100090004032C0D0C0E0C2CF0541E5646009E563ED
:1000A000600575630001B0756301E52360021523E7
:1000B000D0E0D0D032C2AF53E67F7592FA7593FF8D
:1000C000C22053917FD2AF32C2AF53E6EFC0D0C04F
:1000D000E0C0F0D2D3D2AF5388EFA88AA98CAA404F
:1000E000308D010A758A00758C00754000438810B8
:1000F000E564700AC3E833F8E933F9EA33FA3033D8
:100100001FE8C4540FFAE9C454F04AFAC3132AFA98
:10011000C3E833F8E933F9E82AFAE93406FB217336
:1001200030320FC3E833E933FAE82AFAE93400FB46
:100130002173303115E875F056A4AAF0E975F05630
:10014000A42AFAC5F03400FB2173C3EA13FAE913B9
:10015000F9E813F8E875F056A4AAF0E975F056A48A
:100160002AFAC5F03400C313FBEA13FAC3EB13FBFE
:10017000EA13FAC3EB94125006C3EB9406501A0527
:1001800022E52270021522C3E522940A500241C0E2
:100190007552007A007B00418CE522600215223006
:1001A00035067C007D0821B3AC31AD32303A04AC69
:1001B00033AD34C3EA9CFAEB9DFB9208AE5EAF5FB1
:1001C000303A425007203409D23421D1303402C2AF
:1001D00034303404AE60AF61203902B234C3EA3344
:1001E000FAEB33FBA208500AEAF42401FAEBF434E8
:1001F00000FBC3EA9450FAEB9400FB501478007AA9
:10020000007B004111A208500878007A007B004171
:1002100070E5255403601B202A18E55B33F9EB7069
:1002200007C3E99A4002E9FAE53CC4332AFAEB3401
:1002300000FBEA8EF0A4F9AAF0EB8EF0A42AFAC52E
:10024000F03400FBC3EB13FDEA13F8C3ED13FDE834
:1002500013F80FEF146004C3E833F8C3E933EA334B
:10026000FAEB33FBDFEDEB30E30678FF7AFF7B0739
:100270008852D230C3E559FC955A4002AC5AC3ECBF
:1002800095525008EC75F008A4FAABF0EAF4F8EBDC
:10029000F45407F98854895575230AE55830E2105B
:1002A000D0F0D0E0D0D053F7DF43F74043E6103230
:1002B000D0F0D0E0D0D053D8FE43DA0143E610327C
:1002C00075230AD0F0D0E0D0D043E61032C2AF534D
:1002D000A8FEC0D0C0E0D2D38554FB8555FC85551F
:1002E0005853F7BF53DAFEC3E552940140057553E6
:1002F0000041FEE5532401F55350037553FF53F7B6
:10030000DF53D8FED0E0D0D043A801D2AF3279017C
:10031000801479038010790A800C791E8008796432
:10032000800479C880007817E4D5E0FDD8FAD9F6C2
:10033000227A147B7880127A107B8C800C7A0D7B69
:10034000B480067A0B7BC88000E562D5E001227993
:1003500002E4C293D5E0FDD292D293D5E0FDC293E0
:10036000D5E0FDC292D293D5E0FDE920E004D29021
:10037000D29130E004D294D295E562D5E0FDE92037
:10038000E002C29130E002C2957496D5E0FDD9C179
:10039000EAF8D5E0FDD8FBDBB0C2932278FF202835
:1003A0002879A1E76023E548601F74FF8548F08441
:1003B000853FF030290375F005A4F8C5F060027898
:1003C000FFC3E8955B5002A85B885A22C3E54794B7
:1003D000A0E5489400E55A50031461DD046002F57D
:1003E0005A2275E89022055CC3E55C9408405330BE
:1003F000EDF4A8BDA9BE755C00E9FA79A0E76041FB
:10040000EA7006E55D6018800CC3E8955D600EE556
:100410005D5005600A1480070460FA8002E55DF50E
:100420005DC39567401B7559C0C39404401375594B
:1004300080C39404400B755940C39404400375591C
:100440000022E5592410500274FFF55922743279C4
:10045000A687F0A4C5F0A2F733F8C3E89559400287
:10046000A859885B227547007548F022C2AF75C84D
:1004700000A8CCA9CDAA4130CF010A75C804D2AFDB
:10048000C3EA13FAE913F9E813F8AB42AC43884224
:100490008943C3E89BF8E99C20280A547FF9302C53
:1004A00002A18981E3AD448A44F9EA9D547FFA6050
:1004B0000478FF79FFAE45AF468B458C46A842A92C
:1004C00043C3E89EF8E99FF9C3E54813FBE54713EA
:1004D000FAE82AF547E93BF54850067547FF7548A5
:1004E000FFA130AA47AB48AC47AD487E047F02C3AA
:1004F000EB9404400D1E1FC3EB9408400520290215
:100500001E1FC3ED13FDEC13FCDEF7C3EA9CFAEBF0
:100510009DFBEF6009C3E913F9E813F8DFF7EA2858
:10052000FAEB39FB8A478B4850067BFF8B478B4899
:10053000C3EB94025002D22C3028047F03A15B78D5
:1005400092E6FFC3E53D948240110FC3E53D94A0C0
:1005500040010FC3EF940640027F057E02E548C4C8
:10056000540FF9E548C454F0F8E547C4540F28F88F
:10057000C3E89EFAE99400FB4009C3EA9401EB94B6
:100580000050047A01E4FBA1D5AA47AB48EBC4FEB6
:10059000EAC4540F4EFCC3EA9CFAEB9400FBC3E898
:1005A00013C313F8EA28FAEB3400FB8A478B48C3DD
:1005B000EB94024002C22C7802EBC4FE7B00EAC43A
:1005C000540F4EFAC3EA98FA4005C3940150027AD8
:1005D000017892E6FF302002A1D5854E92854F9397
:1005E000D22043E680C3E49AF8E49BF9C3E833F8E9
:1005F000E933F9302C02C167E8FAE9FBD3E913FDCE
:10060000E813FC884E894FC3EF94036037EF20E076
:100610000CE82CF8E93DF9ECFAEDFB8013E828F83A
:10062000E939F9C3E82401F8E93400F97AFF7BFFDE
:10063000C3EF9403400E8A508B51884A894B8C4CEF
:100640008D4DC19B885089518A4A8B4B8C4C8D4D66
:100650003028127550F07551FF754CF0754DFF75CF
:100660004EF0754FFFC19BE8FAD3E813FC884EC3E8
:10067000EF94036020EF20E007E82CF8ECFAC18744
:10068000E8282401F87AFFC3EF940340088A5088D1
:100690004A8C4CC19B88508A4A8C4C302002C19BAA
:1006A000753A02D22043E680E5255403602DA84721
:1006B000A948C3E913F9E813F8302804E92440F9FC
:1006C000C2AF53E67F759100C3E498F594E499F5C1
:1006D00095759104D22043E680D2AF22D22175498C
:1006E00000752000302B03752040800ED221754903
:1006F00000752040302B0375200078017901202CF3
:1007000020E52554036002C2217914E548C3137023
:100710000104F8C3941440027814302804781B793B
:100720001BC3E833F8C3E933F9202010E549600C16
:10073000302803D53A04D223E1B0D1A30549E59B83
:100740005440B52002E19A30280908C3E8994001D5
:1007500018E12920210A08C3E8994002C1FAE129D9
:10076000C221C2AF53E67F759100302C1275940000
:100770007595F0759104D22043E680D2AFC1FAE5B9
:10078000487EFFC3334009C3334005C3334001FEF5
:10079000C3E49E759400F595E173C3E53994015067
:1007A00002C1FA302102C1FAD802E1AEE129C22326
:1007B000C2AF53E67F759100855094855195759130
:1007C00004854A92854B93D22043E680D2AFE5253B
:1007D000540360072029020539801030230D202B97
:1007E0000A20210715811581020F1F227800302170
:1007F000027801E53D75F007A4F9E5F028F5F0E988
:10080000A2F013A2F113A2F213F53DC394785003A2
:10081000753D78C3E53D953E400BD222C291C2930F
:10082000C29575D53F3020020125854C92854D93A8
:10083000D22043E68022203814C2AFC293C290D2A5
:1008400091D29575D52FD2AF759F20213AC2AFC2F4
:1008500093C294D295D29175D53ED2AF759F202187
:100860003A203815C2AFC295D29375D53BC290D20B
:1008700091D2AF759F3002093AC2AFC291D293753F
:10088000D53BC294D295D2AF759F1002093A203859
:1008900014C2AFC291C294D295D29375D53BD2AF58
:1008A000759F10213AC2AFC295C290D291D2937572
:1008B000D53BD2AF759F30213A203815C2AFC293D5
:1008C000D29175D53EC294D295D2AF759F200209C0
:1008D0003AC2AFC293D29575D52FC290D291D2AF02
:1008E000759F2002093A203814C2AFC295C292D235
:1008F00093D29175D53ED2AF759F30803DC2AFC2C5
:1009000091C292D293D29575D52FD2AF759F108098
:1009100029203814C2AFC291D29575D52FC292D278
:1009200093D2AF759F108012C2AFC295D29175D588
:100930003EC292D293D2AF759F30C22222C291C2E0
:1009400093C295C291C293C29575D53F22788076A5
:10095000FF0876FF0876FF0876FF0876FF0876FF27
:100960000876090876FF087601788C76010876FF0C
:100970000876FF0876FF0876FF0876FF08760308FA
:1009800076FF0876FF0876FF0876250876D0087689
:10099000280876500876040876FF0876020876FF65
:1009A00008767A0876FF0876070876010876FF0849
:1009B00076FF08760008760022FA75F00CA4ABF0FA
:1009C000EAC333F8740133F9E8C333F8E933F9E8DB
:1009D000C32BF8E93400F9E8C333F8E933F9227896
:1009E00088E6C39403D23A5002C23AC238E630E1F4
:1009F00002D238A23892397886E614900080937833
:100A0000A6F67886E6F53FC394025003753F027858
:100A10009CE6753EFFB40203753EA0B40303753E29
:100A20008278A0E6F8600674282409D8FCF5677877
:100A300096E631B988318932789EE631B9883389B2
:100A4000347897E631B988358936313D2230351111
:100A50007A007B007CFF7D007E0051B48B5F8A5E54
:100A600022303A227896E6FA7B00789EE6FC7D00FA
:100A7000C3EA33FAEB33FBC3EC33FCED33FD7E0A00
:100A800051B48B618A607896303A02789EE6FA7BA0
:100A9000007897E6FC7D007E00303A10C3EA33FA16
:100AA000EB33FBC3EC33FCED33FD7E0A51B48B5FBB
:100AB0008A5E2222C3EC9EFCED9400FDC3EC9AFCFE
:100AC000ED9BFDC3EC9423ED940050047C237D004A
:100AD000C3EC94FFED940140047CFF7D017BFF0B90
:100AE0007A000AEA7009C3EC33FCED33FD41DFEC18
:100AF0008AF0A4AEF0ED8AF0A42E947C40E4EAF4EF
:100B000060DD22D235514D12031A12031A7A007B8E
:100B1000007C10120312E5522AFA74003BFBDCF34E
:100B20007C04C3EB13FBEA13FADCF7FFEB60027FF4
:100B3000FFC235514D2278A5E6F954037000E954FF
:100B40000C7000E954307000E954C07000227565E3
:100B5000007566007597DE7597AD7581C043FF809F
:100B600075EF0675A900313D7580FF75F1F075A42C
:100B7000007580FF75D4FF75900075F23F75A53F35
:100B800075900075D53F75A60175E34075E2023199
:100B90003DE4F8F6D8FD314DF166789886627530FF
:100BA00001C2AF12032212033112031A12033712C9
:100BB000031A12033D12031A7136C2AF7565007530
:100BC000660078FA79FA308507D9FBD8F7021C005D
:100BD00031DF514D78988662313D75A91375A710A4
:100BE00075C10075A70075640075E40575881175F9
:100BF0008E0475890975C80475910475D84075D936
:100C00000875F783759E0075960275DA4A75DB00E4
:100C100075A82375E69075F310759B80759D00751A
:100C2000D10C75BCB975BB1075E88075B2011203A3
:100C30000ED2AF753C00C230120322C231752200C1
:100C400012031EC3E522940A4024D231C232752217
:100C50000012031EC3E522940A4013D232C2337538
:100C6000220012031EC3E522940A4002D23312036B
:100C700012203003020BBAC2AF1203311203311239
:100C80000331D2AF120322303A02A12C12031278A0
:100C90008CE6C394015002A12CE530C394015002AC
:100CA000A12C7565A57566F17F02D235514D1203F1
:100CB0001EC2AFC235514DC3E552947FD2AF406CD6
:100CC00012030EC2AF120343D2AFDFDE7103C3EFD4
:100CD0007897F612032212104E7F0AD235514D1228
:100CE000031EC2AFC235514DC3E552947FD2AF50FF
:100CF000E812030EC2AF120331120316120331D2EF
:100D0000AFDFD87103EF24037896F6F87997E7C33D
:100D100094234003985006E824237897F612032280
:100D2000F1A012107D12031E514D61BA7565007558
:100D3000660012031E7801303A027805C3E5529826
:100D400040028187C2AF120343120343120343D20E
:100D5000AF120322753000E4F537F5380537E53773
:100D6000F4703E0538789AE67819146012783214D7
:100D7000600D787D14600878FA146003753800C33C
:100D8000E53898401C313D12030E15387537007850
:100D9000998662C2AF120343D2AF7898866212037B
:100DA0001E120316E523700261BA7801C3E552985A
:100DB00040AA12031EE5237003020BBAC2AF313DF5
:100DC000E4D2AFE4F55CF524F525F53D755C081239
:100DD000030E1203E230EDFDA8BDA9BEE97001F8D3
:100DE000885D1203E6755C08C2AF7559FF12044DA9
:100DF000855B59855B5AD2AF75A71075C13075A751
:100E00000075A903756401303A07C238303402D244
:100E100038D22875390011E6311112046512046CBC
:100E200012046512046C1204651206EC1207EC1130
:100E30003612046C1206DC202C0312039C302C03A7
:100E40001203CC1207EC116112046C1206EC1207AB
:100E5000EC118E12046C1206DC1207EC11B91204AC
:100E60006C1206EC1207EC11E612046C1203E2128B
:100E700006DC1207EC31111203E612046C3028274D
:100E8000855B5979187A0CC3E53999400EC228D28E
:100E9000298A3B855B59855B5A800CC3E5529401D6
:100EA0004003020E29E12730291C202B19E53B14B1
:100EB0007006C229D22AC129F53BC3E552940140EC
:100EC00003020E298061753C0078FA79A4E760027C
:100ED0007803C3E55398504FE523604B303A172011
:100EE0003805203407800F303402800A202B07D2C7
:100EF0002B855B59C15678F0302B05855B597820DE
:100F0000C3E548985003020E29302B1BC22BC23870
:100F1000303402D238D229753B12855B59C129057C
:100F20003CE5526002E12A753C00C2AF313D7524B8
:100F30000075250075A91375A71075C10075A70068
:100F4000756400D2AF12031E313D78A4E6600CC276
:100F500090D291C292D293C294D295C3E53C9404AC
:100F6000400261BAA157901A0D7820F1DDE520B456
:100F7000550AA3F1DDE520B4AA028006314DF1A0A7
:100F8000801D901A0378807B0AF1DDA308DBFA90BC
:100F90001A0F788C7B1AF1DDA308DBFA901A29224C
:100FA000C2AF121022120FFD901A007410F1E2A3CA
:100FB0007403F1E2A37421F1E2901A0378807B0AB2
:100FC000F1E1A308DBFA901A0F788C7B1AF1E1A308
:100FD00008DBFA121036121011901A2922E493F647
:100FE00022E6438F01538FFDFFC3E583941C40012C
:100FF00022EF8565B78566B7F0538FFE22438F02D7
:10100000438F018565B78566B7901A0DF0538FFC45
:1010100022901A0D7455120FE2901A0E74AA120F34
:10102000E2227A3079D07820901A40120FDDE52044
:10103000F709A3DAF6227A3079D0901A40E7120F36
:10104000E209A3DAF8227C05120322DCFB22C2AFFC
:1010500012033112033712033D1203431203161217
:10106000033112033712033D120343120316120316
:101070003112033712033D120343D2AF22C2AF1223
:10108000034312033D1203371203311203161203F6
:101090004312033D120337120331120316120343A6
:0C10A00012033D120337120331D2AF22BD
:1019FD00020B4E100321FFFFFFFFFFFF09FF01FF49
:101A0D0055AA01FFFFFFFFFF03FFFFFF25D0285061
:0D1A1D0004FF02FF7AFF0701FFFF0000FF3A
:101A400023415F485F3030232020202020202020A9
:101A500023424C48454C492445464D3842323123B7
:101A60002020202020202020202020202020202076
:101C0000C2AFC2D37597DE7597AD7581C075A90057
:101C100043FF80752438752503B1DB7529A5752A26
:101C2000F143F12053A4DFD28575D4FF75E3407DE5
:101C3000FA780379E67C10752200752300901DE880
:101C40007B0675249875250130850281482085081A
:101C5000D8FBD9F9DCF781BA308508D8FBD9F9DC93
:101C6000F781BAB19BE493A3C39A6004DDC381BA40
:101C7000DBDBB18D600281317B08E493FAA3B16EA6
:101C8000DBF87A30B16E752200752300B18DEAFC65
:101C9000EBFDC3ED94FE400EB18D8A278B28ED300D
:101CA000E0048A828B83B18D7AC270D8C3ED94FE32
:101CB000601950CEBD0029EC600F7520007521FF22
:101CC000752900752A000200008100A827A92808AC
:101CD00009D804D90281DDB191EAF281D10D81A642
:101CE000C3ED94035051EDA2E092007AC5C3E582A2
:101CF0009400E583941C508C200010438F02438F86
:101D0000018529B7852AB7F0300027A827A9280818
:101D100009438F01538FFDD804D902A132C3E58353
:101D2000941C4003A3A117E28529B7852AB7F0A325
:101D3000A117538FFC81827AC1BD030CE493A3FAEF
:101D4000B152DCF8B14A81828184AA22AB23B16E00
:101D5000EBFAEA6222752608C3E52313F523E52290
:101D600013F52250066323A0632201D526EAB1DBD6
:101D7000B1DB75260AEAF4200102D285300102C2E5
:101D800085B1DBC3134002C201D526EB22B191EA33
:101D9000FB208502A191308502A196752608AE240C
:101DA000AF25C3EF13FFEE13FEB1DFB1DBC3EA13C0
:101DB0003085024480FA30E703632201C3E5231330
:101DC000F523E52213F52250066323A0632201D5F3
:101DD00026D9E52265236523F52222AE24AF250E00
:101DE0000FDEFEDFFCD20122424C48656C693437BD
:061DF0003163E8B20601B8
:00000001FF
